:020000020000FC
:020000000BC033
:02001200E8C044
:10001600D4C00FE50DBF02E00EBF08E90AB907E03C
:1000260009B900E00ABB0FEF0BBB00E007BB0FEFFF
:1000360008BB0FEF04BB05BB01BB02BB02E6402EAB
:10004600502E02E9202E302EA7D0789400E0602EA4
:1000560002EA702EF2E0ECE40EEF31D00DEF2FD075
:100066000BEF2DD007EF2BD00FEE29D00FED27D0B9
:100076000FEB25D00FE723D00EEF2BD00DEF29D0B5
:100086000BEF27D007EF25D00FEE23D00FED21D0B1
:100096000FEB1FD00FE71DD00FEE25D00FED23D0AD
:1000A6000FEB21D00FE71FD00FEE27D00FED25D095
:1000B6000FEB23D00FE721D00EEFB9D0C7CF05BB8A
:1000C6000FEF02BB0000000000000000000039B383
:1000D6001EC005BB0FEF02BB0000000000000000C1
:1000E600000036B314C002BB0FEF05BB00000000D2
:1000F60000000000000039B30AC002BB0FEF05BBC9
:100106000000000000000000000036B300C030957B
:10011600B62DA72D4D915C915F933E930D9143278C
:10012600052F04234095532F5423502B5D934F9155
:100136004527352F6B2E7A2E68E0479570F0379558
:10014600C895002D31960E3FD9F7C895002D3196EA
:100156000E3FD9F76A9589F70895379538F0C8950F
:10016600002D31960E3FD9F708D0F4CF06D0C895AA
:10017600002D31960E3FD9F7EDCFC895002D31965B
:100186000D3F29F00E3F11F052D0F7CF08950F9191
:100196000F910F910F9158CF02EAB0E0A02F00E423
:1001A60020E02D930A95E9F708951FB71F930F9343
:1001B6000F911FBF1F911FBF18951FB71F93569A08
:1001C600451411F4569808C0C42DD0E019911CB9F5
:1001D600C23909F4C2E64C2E1F911FBF18951FB7EE
:1001E6001F931CB1109361005C99F6CFC22DD0E02D
:1001F6001993C23A09F4C2E92C2E231431F433942C
:10020600132D123A11F412E9312E122D13190AF494
:10021600105F10936000E0CF231409F4FDCFA32DE7
:10022600B0E00D91A23A09F4A2E93A2E0895B0E0A1
:10023600A52D0D93A23909F4A2E6A415F1F35A2EC1
:10024600569BBBDF089590247FFE80247FFE902579
:100256007FFE80257FFE90267FFE80267FFE9027EC
:100266007FFE80277FFE90287FFE80287FFE9029D4
:100276007FFE80297FFE902A7FFE802A7FFE902BBC
:100286007FFE802B7FFE902C7FFE802C7FFE902DA4
:100296007FFE802D7FFE902E7FFE802E7FFE902F8C
:1002A6007FFE802F7FFE90307FFE80307FFE903174
:1002B6007FFE80317FFE90327FFE80327FFE90335C
:1002C6007FFE80337FFE90347FFE80347FFE903544
:1002D6007FFE80357FFE90367FFE80367FFE90372C
:1002E6007FFE80377FFE90387FFE80387FFE903914
:1002F6007FFE80397FFE903A7FFE803A7FFE903BFC
:100306007FFE803B7FFE903C7FFE803C7FFE903DE3
:100316007FFE803D7FFE903E7FFE803E7FFE903FCB
:100326007FFE803F7FFE90407FFE80407FFE9041B3
:100336007FFE80417FFE90427FFE80427FFE90439B
:100346007FFE80437FFE90447FFE80447FFE904583
:100356007FFE80457FFE90467FFE80467FFE90476B
:100366007FFE80477FFE90487FFE80487FFE904953
:100376007FFE80497FFE904A7FFE804A7FFE904B3B
:100386007FFE804B7FFE904C7FFE804C7FFE904D23
:100396007FFE804D7FFE904E7FFE804E7FFE904F0B
:1003A6007FFE804F7FFE90507FFE80507FFE9051F3
:1003B6007FFE80517FFE90527FFE80527FFE9053DB
:1003C6007FFE80537FFE90547FFE80547FFE9055C3
:1003D6007FFE80557FFE90567FFE80567FFE9057AB
:1003E6007FFE80577FFE90587FFE80587FFE905993
:1003F6007FFE80597FFE905A7FFE805A7FFE905B7B
:100406007FFE805B7FFE905C7FFE805C7FFE901DA2
:100416007FFE801D7FFE901E7FFE801E7FFE901F4A
:100426007FFE801F7FFE90207FFE80207FFE902132
:100436007FFE80217FFE90227FFE80227FFE90231A
:100446007FFE80237FFEB07B00FEC010FDFEB07BEA
:1004560000FEC012FDFEB07B00FEFE0091277FFE6F
:1004660081277FFE91287FFE81287FFE91297FFECE
:1004760081297FFE912A7FFE812A7FFE912B7FFEB6
:10048600812B7FFE912C7FFE812C7FFE912D7FFE9E
:10049600812D7FFE912E7FFE812E7FFE912F7FFE86
:1004A600812F7FFE91307FFE81307FFE91317FFE6E
:1004B60081317FFE91327FFE81327FFE91337FFE56
:1004C60081337FFE91347FFE81347FFE91357FFE3E
:1004D60081357FFE91367FFE81367FFE91377FFE26
:1004E60081377FFE91387FFE81387FFE91397FFE0E
:1004F60081397FFE913A7FFE813A7FFE913B7FFEF6
:10050600813B7FFE913C7FFE813C7FFE913D7FFEDD
:10051600813D7FFE913E7FFE813E7FFE913F7FFEC5
:10052600813F7FFE91407FFE81407FFE91417FFEAD
:1005360081417FFE91427FFE81427FFE91437FFE95
:1005460081437FFE91447FFE81447FFE91457FFE7D
:1005560081457FFE91467FFE81467FFE91477FFE65
:1005660081477FFE91487FFE81487FFE91497FFE4D
:1005760081497FFE914A7FFE814A7FFE914B7FFE35
:10058600814B7FFE914C7FFE814C7FFE914D7FFE1D
:10059600814D7FFE914E7FFE814E7FFE914F7FFE05
:1005A600814F7FFE91507FFE81507FFE91517FFEED
:1005B60081517FFE91527FFE81527FFE91537FFED5
:1005C60081537FFE91547FFE81547FFE91557FFEBD
:1005D60081557FFE91567FFE81567FFE91577FFEA5
:1005E60081577FFE91587FFE81587FFE91597FFE8D
:1005F60081597FFE915A7FFE815A7FFE915B7FFE75
:10060600815B7FFE915C7FFE815C7FFE911D7FFE9C
:10061600811D7FFE911E7FFE811E7FFE911F7FFE44
:10062600811F7FFE91207FFE81207FFE91217FFE2C
:1006360081217FFE91227FFE81227FFE91237FFE14
:1006460081237FFE92247FFE82247FFE92257FFEF9
:1006560082257FFE92267FFE82267FFE92277FFEE0
:1006660082277FFE92287FFE82287FFE92297FFEC8
:1006760082297FFE922A7FFE822A7FFE922B7FFEB0
:10068600822B7FFE922C7FFE822C7FFE922D7FFE98
:10069600822D7FFE922E7FFE822E7FFE922F7FFE80
:1006A600822F7FFE92307FFE82307FFE92317FFE68
:1006B60082317FFE92327FFE82327FFE92337FFE50
:1006C60082337FFE92347FFE82347FFE92357FFE38
:1006D60082357FFE92367FFE82367FFE92377FFE20
:1006E60082377FFE92387FFE82387FFE92397FFE08
:1006F60082397FFE923A7FFE823A7FFE923B7FFEF0
:10070600823B7FFE923C7FFE823C7FFE923D7FFED7
:10071600823D7FFE923E7FFE823E7FFE923F7FFEBF
:10072600823F7FFE92407FFE82407FFE92417FFEA7
:1007360082417FFE92427FFE82427FFE92437FFE8F
:1007460082437FFE92447FFE82447FFE92457FFE77
:1007560082457FFE92467FFE82467FFE92477FFE5F
:1007660082477FFE92487FFE82487FFE92497FFE47
:1007760082497FFE924A7FFE824A7FFE924B7FFE2F
:10078600824B7FFE924C7FFE824C7FFE924D7FFE17
:10079600824D7FFE924E7FFE824E7FFE924F7FFEFF
:1007A600824F7FFE92507FFE82507FFE92517FFEE7
:1007B60082517FFE92527FFE82527FFE92537FFECF
:1007C60082537FFE92547FFE82547FFE92557FFEB7
:1007D60082557FFE92567FFE82567FFE92577FFE9F
:1007E60082577FFE92587FFE82587FFE92597FFE87
:1007F60082597FFE925A7FFE825A7FFE925B7FFE6F
:10080600825B7FFE925C7FFE825C7FFE921D7FFE96
:10081600821D7FFE921E7FFE821E7FFE921F7FFE3E
:10082600821F7FFE92207FFE82207FFE92217FFE26
:1008360082217FFE92227FFE82227FFE92237FFE0E
:0408460082237FFE8C
:00000001FF
